:100000000C944A000C9467000C9467000C946700F1
:100010000C9467000C9467000C9467000C946700C4
:100020000C9467000C9467000C9467000C946700B4
:100030000C9467000C9467000C9467000C946700A4
:100040000C9467000C9467000C9467000C94670094
:100050000C9467000C9467000C9467000C94670084
:100060000C9467000C9467000C9467000C94670074
:100070000C9467000C9467000C9467000C94670064
:100080000C9467000C9467000C9467000C94670054
:100090000C94670011241FBECFEFD0E1DEBFCDBFAF
:1000A00011E0A0E0B1E0E6EAF2E000E00BBF02C040
:1000B00007900D92A030B107D9F711E0A0E0B1E0B0
:1000C00001C01D92A030B107E1F70C9418010C9407
:1000D0000000CF93DF93CDB7DEB7109222001092CD
:1000E00021001092250010922400109228001092F6
:1000F000270010922B0010922A0080E180932E009E
:1001000082E180932D001092310010923000DF9137
:10011000CF910895CF93DF93CDB7DEB788E1809379
:10012000600087E080936000DF91CF910895CF93C6
:10013000DF93CDB7DEB726970FB6F894DEBF0FBEBC
:10014000CDBF69837A838B839C8389819A81AB81BC
:10015000BC819C01AD01689413F8220F331F441F2A
:10016000551F1694D1F780E094E2A4EFB0E0BC01F3
:10017000CD010E943101DA01C90101979E838D836F
:100180008D819E81892F99278093C5008D818093D1
:10019000C40088E18093C10086E08093C200269667
:1001A0000FB6F894DEBF0FBECDBFDF91CF9108959B
:1001B000CF93DF93CDB7DEB722970FB6F894DEBFAB
:1001C0000FBECDBF8091C000882334F48091C6005B
:1001D00099279A83898302C01A82198289819A8118
:1001E00022960FB6F894DEBF0FBECDBFDF91CF9140
:1001F0000895CF93DF93CDB7DEB721970FB6F8946C
:10020000DEBF0FBECDBF89838091C0009927807269
:100210009070009709F4F8CF89818093C6002196E9
:100220000FB6F894DEBF0FBECDBFDF91CF9108951A
:10023000CEEFD0E1DEBFCDBF0E948A000E946900F0
:1002400060E875E280E090E00E949700A8950E9427
:10025000D800898389818823C9F389810E94F900A4
:10026000F5CFA1E21A2EAA1BBB1BFD010DC0AA1FD0
:10027000BB1FEE1FFF1FA217B307E407F50720F00F
:10028000A21BB30BE40BF50B661F771F881F991F8A
:100290001A9469F760957095809590959B01AC01D3
:0602A000BD01CF0108952D
:00000001FF
